:05893F0033302E38006A
:106DCA00C105C100C104C102C103C1014109355E47
:1083D100AE8475840F75A40F7580F075A7F0E4FD68
:1083E100FC0DBD00010CBC4EF8BD20F5E58030E66A
:1083F10004E4FF800CE5B0540F70047F018002E4B7
:03840100FF8E8467
:018404002255
:10409A00900765124C2000000000E4900769F09038
:1040AA00076BF090076FF0A3F075FFDE75FFAD1296
:1040BA0086A2900935E0FF1288B043F602D2AFC259
:1040CA0004E49006A4F01284A0E4900771F090072B
:1040DA0071E0FFD39403500DE4FD128894900771A8
:1040EA00E004F080E975840F128286128524900616
:1040FA00A8E0FCA3E0FDE4FF12773E9006ADE0FCE9
:10410A00A3E0FD7F0112773E9006B2E0FCA3E0FD3A
:10411A007F0212773E9006B7E0FCA3E0FD7F031210
:10412A00773ED205D20075840F125B41900796E064
:10413A00B4011712745190076AEFF0E02492F582E5
:10414A00E43407F5837401F0800690076A74FFF07F
:10415A00900796E06401703E90076AE0FF12846D52
:10416A0090076CEBF0A3EAF0A3E9F01248BAB402A4
:10417A000A90076AE0FF12706D801B90076CE0FBE3
:10418A00A3E0FAA3E0F91248BAB4010A90076AE078
:10419A00FF7D01127345E4900771F0900771E0FF0B
:1041AA00D39403400302423590076AE0FEEF6E6043
:1041BA007A900771E0FF12846D90076CEBF0A3EA26
:1041CA00F0A3E9F0900771E0FF2492F582E4340746
:1041DA00F583E06401703390076CE0FBA3E0FAA377
:1041EA00E0F91248BAB4020512706D803590076C76
:1041FA00E0FBA3E0FAA3E0F91248BAB4012490075D
:10420A0071E0FFE4FD127345801890076CE0FBA390
:10421A00E0FAA3E0F91248BA7008900771E0FF12B9
:10422A0071A0900771E004F00241A51286FBEF70BD
:10423A000302455F127F74EFB4190040030245512F
:10424A00904251F828287302429C0242D20242D676
:10425A000242DA0242DE0242E60242EA0242EE0288
:10426A0042F20242FA02437F0243940243A002430B
:10427A00D70244130244750244EF0244FD0245107A
:10428A0002451C0245280245390242C102454F0235
:10429A00438F300215A204B39204300409C20ED22D
:1042AA0003128734800CC20380083003051289394F
:1042BA00C203D205024551900935E0FF7BFF7A8996
:1042CA00793F127C8C024551E4FF800A7F01800607
:1042DA007F0280027F031273CC024551E4FF800AF9
:1042EA007F0180067F0280027F031287E202455126
:1042FA009006A7E00490078BF090078BE0C3941513
:10430A00502BE0FF25E024DAF582E43406F583E059
:10431A00FCA3E0FDEF25E024D8F582E43406F5831A
:10432A00ECF0A3EDF090078BE004F080CC128367E9
:10433A00900702EEF0A3EFF01287189006A7E02587
:10434A00E024DAF582E43406F583E0FFA3E0900680
:10435A00A8CFF0A3EFF09006A7E025E024DAF582D3
:10436A00E43406F583E0FCA3E0FDE4FF12773E1295
:05437A0082C002440CAA
:10437F00300105127A9BC20112639E128718807D4D
:10438F00D20102446E9006BDE0F4F012873402446D
:10439F006E9006A7E0D3940050030245519006A7F4
:1043AF00E014F0E025E024DAF582E43406F583E04A
:1043BF00FEA3E0FF9006A8EEF0FCA3EFF0FDE4FFF4
:1043CF0012773E12873480359006A7E0C3941440CD
:1043DF00030245519006A7E004F0E025E024DAF54A
:1043EF0082E43406F583E0FEA3E0FF9006A8EEF02A
:1043FF00FCA3EFF0FDE4FF12773E128734D200D218
:10440F0005024551D39006A9E094269006A8E094A2
:10441F002A4007742AF0A37426F0D39006A9E094DB
:10442F002E9006A8E094225003024551A3E024F6F3
:10443F00F09006A8E034FFF09006A8E0FCA3E0FDA2
:10444F009006A7E025E024DAF582E43406F583EC44
:10445F00F0A3EDF0E4FF12773E1279C8128734D241
:10446F0005D2000245519006A8E07002A3E0700A41
:10447F009006A87422F0A3742EF09006A8E0FEA375
:10448F00E0FFC3942EEE9422500C9006A87422F0F5
:10449F00A3742EF0801AD3EF941CEE942A400302DB
:1044AF0045519006A9E0240AF09006A8E03400F0E8
:1044BF009006A8E0FCA3E0FD9006A7E025E024DA33
:1044CF00F582E43406F583ECF0A3EDF0E4FF127708
:1044DF003E1279C8128734D205D200128734806217
:1044EF002001047F018037900704E014800C200125
:1044FF00047F01803A900704E004F0E0547FF080DD
:10450F00412001047F0280169007058019200104C5
:10451F007F02801B900705801E2001077F03126A10
:10452F00B6801F900706E014800F2001077F03124B
:10453F006900800E900706E004F0E0540FF080024F
:10454F0080FE300102D2001286FBEF600302423E72
:10455F007B017A0779721284CDEF70030247AE9018
:10456F000774E0124C5145E804462F0545A6144543
:10457F009416459D1745AF1A45D11B45DC1D45E2E5
:10458F001E0000467CD204D203D20502467CC20430
:10459F00C203D20502467CD202D204D20302467C69
:1045AF007B017A077972900782EBF0A3EAF0A3E917
:1045BF00F01248BAFE900935E0FF6E600302467CA8
:1045CF008005900935E0FF12862302467C1289147C
:1045DF0002467C12893302467C7B017A07797290FE
:1045EF000785EBF0A3EAF0A3E9F09000031248D39C
:1045FF00FF900935E06F707530046A90078504F0FD
:10460F00A3EAF0A3E9F09000051248D3FF9000064B
:10461F001248D3FD9000041248D3FB124F7080450F
:10462F007B017A077972900785EBF0A3EAF0A3E993
:10463F00F09000031248D3FF900935E06F702E30D1
:10464F00042390078504F0A3EAF0A3E9F090000596
:10465F001248D3FF9000061248D3FD900004124871
:10466F00D3FB126D17900935E0FF12866520040306
:10467F0002455F900774E014603524FA605514709A
:10468F000302472E240660030247621288457B010E
:10469F007A077972900782EBF0A3EAF0A3E9F09022
:1046AF0000031248D39006A4F012893902475F7BAA
:1046BF00017A077972900782EBF0A3EAF0A3E9F091
:1046CF009000031248D39006A4F090076B7401F08A
:1046DF000247621288457B017A077972900788EB4F
:1046EF00F0A3EAF0A3E9F09000031248D3FF900083
:1046FF00041248D3FD9000051248D3FBC003900766
:10470F0088E0FBA3E0FAA3E0F99000061248D390EB
:10471F000808F0D0031269DC90076BEFF0803112BC
:10472F0088457B017A077972900788EBF0A3EAF04E
:10473F00A3E9F09000031248D3FF9000041248D36E
:10474F00FD9000051248D3FB12597690076BEFF0DE
:10475F001288CA90076BE0700302455F12852490A0
:10476F0006A8E0FCA3E0FDE4FF12773E9006ADE063
:10477F00FCA3E0FD7F0112773E9006B2E0FCA3E0C0
:10478F00FD7F0212773E9006B7E0FCA3E0FD7F03AA
:10479F0012773ED200D205E490076BF002455F30EE
:1047AF0005051260EEC205200003024130126C5A5B
:0547BF00C200024130C0
:0350330002819A5D
:10819A00C0E0C0F0C083C082C0D075D000C000C0AB
:1081AA0001C002C003C004C005C006C007C2CF1286
:1081BA004CA3D007D006D005D004D003D002D001FA
:0D81CA00D000D0D0D082D083D0F0D0E032F1
:10809300AB84A2AF9209E4FCFDED9008E1124C140D
:1080A3009008E3E0FEA3E07811A60608F6E4F58461
:1080B300C2AF43B701438F02438F0118E6FE08E6C0
:1080C300F5828E83E4F053B7FEF58FA20992AFAF2A
:0380D300038F8494
:0180D6002287
:027DF200AB05DF
:107DF400AA84A2AF920AE4FCFDED9008E5124C14AB
:107E0400EBFF3395E0FEEFF44E60299008E7E0FEC7
:107E1400A3E07813A60608F6E4F584C2AF43B701DD
:107E2400758F0118E6FC08E6F5828C83EBF053B7F6
:0C7E3400FEE4F58FA20A92AFAF028F842B
:017E4000221F
:107BCA009008AFEEF0A3EFF0A3ECF0A3EDF0A3EA78
:107BDA00F0A3EBF09008B3E07002A3E060429008D3
:107BEA00AFE0FEA3E0FFA3E0FCA3E0F5828C83E014
:107BFA00FD127DF29008B4E024FFF09008B3E0345F
:107C0A00FFF09008B2E004F070069008B1E004F0CA
:107C1A009008B0E004F070BC9008AFE004F080B4C3
:017C2A002237
:0888FE00E4900000F0A3F02259
:10854D00900000E0FEA3E0FF128093900000E0FE9B
:10855D00A3E0FF7C007D027B007A04127BCAE490CD
:06856D000000F0A3F02263
:0A722D00A9059008B5EEF0A3EFF0FC
:10723700EE54FCFE900000E0FCA3E0FD7002EE6C53
:107247006057ED4C600312854D9008B5E0FEEE5493
:10725700FCFE7F00900000F0A3EFF09008B7EEF07F
:10726700A3EFF0A37400F0A37402F07E049008B7B4
:10727700E475F001124A0685F082F583E493FD90E8
:1072870008B9E475F001124A0685F082F583EDF03E
:10729700EF1F70011EEF4E70D49008B5E0FCA3E01D
:1072A700FDEC5403FC74022DF58274003CF583E970
:0172B700F0E6
:0172B80022B3
:10800800900885EEF0A3EFF0A3EBF0A3EAF0A3E964
:10801800F090088A74FFF5F0124A0645F060269041
:108028000885E475F001124A06AFF0FE900887E073
:10803800FBA3E475F001124A06A9F0FA1248BAFD4A
:0680480012722D80CC2213
:0E804E009008BBEBF0A3EAF0A3E9F0A3EDF07D
:10805C00E49008C0F09008BBE0FBA3E0FAA3E0F9C1
:10806C00A3E0900890F09008BFE0900891F0E4FF36
:10807C001275C9EFB4FF0D9008C0E0FE04F0EEC31A
:06808C00940340D17E00C8
:0180920022CB
:0B84CD0090091DEBF0A3EAF0A3E9F01A
:1084D8007E007F007D10124C7790091DE0FBA3E021
:1084E800FAA3E0F97D101265EFEF7002FF227F0119
:0184F8002261
:107C8C009008357422F0A3EFF0A37413F01248BAE5
:107C9C00900838F09000011248D3900839F0900009
:107CAC00021248D390083AF09000031248D390087F
:107CBC003BF09000041248D390083CF09000051261
:107CCC0048D390083DF09000061248D390083EF03F
:107CDC007B017A087935E49008BFF07D0A02804E6A
:108602009008E97422F0A3EFF0A37403F0A374FFBF
:10861200F07B017A0879E9E49008BFF07D040280DA
:018622004E09
:108623009008ED7422F0A3EFF0A3741CF0A374FF81
:10863300F07B017A0879EDE49008BFF07D040280B5
:018643004EE8
:10866500E49008F1F0A3EFF0A3740AF0A3EFF07B18
:0F867500017A0879F1E49008BFF07D0402804E8D
:106DDA00420522000042040D00004204080000C1DE
:056DEA0008C107C1060D
:0A88EB00C207C208E490040CF0225A
:1085BE00E4900522F0A3F090040DF0A3F0A3F09048
:1085CE000408F0A3F090040304F0A3E4F090040B6D
:0285DE00F02289
:06891B001288EB0285BE8C
:10878300E4F5848FC343C30175C04475CF8EC2C360
:0987930043E60290040A04F022FE
:10884500E4F58420C7FDC2C212891BE490040AF036
:018855002200
:0B88CA00E4F584D2C290040A04F022FE
:0D88B000AE07128783900407EFF002891BCA
:10859900E4900937F0A3F0300702FF222008FDD24A
:1085A90007900405E4F0A37410F0900510EFF0E4CF
:0485B900A3F07F01AB
:0185BD00229B
:1084050030070A900405E07002A3E070037F0022A4
:10841500900406E024FFF0900405E034FFF0900599
:1084250011E0FE04F074122EF582E43405F583EFB5
:04843500F07F0122B1
:0B88D500300707C207D208125009222A
:0E500900AF84E4F58420C7FDC2C4D2C58F84F5
:015017002276
:1075C90090088DEBF0A3EAF0A3E9F090040AE070CB
:1075D90002FF22900890E0FE6005D3941040037FDB
:0875E9000022128599EF604EAB
:1075F100E4900892F0900890E0FF900892E0FEC3BA
:107601009F502490088DE0FBA3E0FAA3E0F98E825D
:107611007583001248D3FF128405EF7002FF229098
:107621000892E004F080CEE490040CF01288D5902A
:0E7631000891E070032008FD90040CE0FF2299
:03763F007FFF22A8
:0E65EF009008F5EBF0A3EAF0A3E9F0A3EDF0BD
:1065FD00E4FFD3900523E09400900522E06480949D
:10660D008050012253E6FD900408E0FEA3E0240F24
:10661D00F58274043EF583E0FF900408E475F00103
:10662D001249F0FCE4B5F00BECB40107E49004085A
:10663D00F0A3F0900404E004F07006900403E0046D
:10664D00F0E4FE9008F8E0FDEEC39D5056EEC39FBA
:10665D005051900408E0FCA3E0240FF58274043C33
:10666D00F583E0FD9008F5E0FBA3E0FAA3E0F98ED9
:10667D0082758300ED124967900408E475F00112EC
:10668D0049F0FCE4B5F00BECB40107E4900408F01C
:10669D00A3F0900404E004F07006900403E004F00D
:1066AD000E80A0EEC39F502B900408E475F00112EC
:1066BD0049F0FCE4B5F00BECB40107E4900408F0EC
:1066CD00A3F0900404E004F07006900403E004F0DD
:1066DD000E80D0900523E024FFF0900522E034FFDA
:1066ED00F043E6029008F8E0FEEFC39E50028002F0
:0266FD00AF06E6
:0166FF002278
:10501B00D3900523E09400900522E06480948040B7
:08502B00047F0180027F0022D6
:03501800025F8EA6
:105F8E00C0E0C0F0C083C082C0D075D000C000C0D9
:035F9E0006C00733
:105FA100C20BAFC1EF124C515FD7085FD7105FE74B
:105FB100185FEC205FF92860263060313860396065
:105FC100603468603970603478604180604190600D
:105FD100BAA0000060C8900510E0F5C2C2C59005E6
:105FE1000FE4F00260CA900511802890040C74FD42
:105FF100F0D2C4D2C50260CA900511E0FF90050F2E
:10600100E0C39F5014E0FF04F074122FF582E434D2
:1060110005F583E0F5C20260CAD2C490040CE4F035
:10602100C2080260CAD2C590040C74FEF00260CAB4
:106031000260BFD2060260CA900402E4F00260CAA4
:10604100900402E07020E5C2F0E0FFC3900404E098
:106051009F7480F8900403E064809850031285BE19
:10606100900402E004F0900404E024FFF0900403A3
:10607100E034FFF090040DE0FEA3E0240FF58274FC
:10608100043EF583E5C2F090040DE475F001124978
:10609100F0FEE4B5F00BEEB4010790040DE4F0A3BB
:1060A100F0900402E014F07020900523E004F070F9
:1060B10018900522E004F0801030060DC20690050C
:1060C1000FE4F0D2C58002D20B300B0EC2C6D2C68D
:0C60D100C2C5C2C4D2C2C20BC208C2C306
:1060DD00D007D006D000D0D0D082D083D0F0D0E081
:0160ED003280
:05892100A2C7E433FFD2
:01892600222E
:06892700C2C253E6FD226E
:105CBA00900853E0FFA3E0FCA3E0FDA3E0FBA3E010
:105CCA00FAA3E0F9900818E50DF0E50EA3F09008A4
:065CDA005BE090081AF0E7
:105CE000900812EFF0A3ECF0A3EDF0A3EBF0A3EA21
:045CF000F0A3E9F044
:105CF40090081B7403F0A374E8F0A3E584F0E4F5C2
:105D04008420C7FDC2C4D2C2D2C5E4FF90094CF0BE
:105D140030C3FDAEC1EE24F8602324F8601F24F8DC
:105D2400602F24F8603624F8603A24F87003025D8A
:105D3400CC24F87003025DD42438025DDCEF700CCF
:105D4400900812E025E044A0F5C27F03C2C5025DBD
:105D5400E2900813E0F5C27F05025DE290094C74FD
:105D640003F0807AEFB4050B900813A3E0F5C27F2B
:105D740006806BEF6406703E90081AE09008157078
:105D84000FE0FBA3E475F001124A06A9F0FA8008BB
:105D9400E0FBA3E0FAA3E0F91248BAF5C2900819AF
:105DA400E024FFF0900818E034FFF0E07002A3E074
:105DB400702C7F078028EFB40706D2C47F09801EA9
:105DC40090094C7405F0801690094C7404F0800E10
:105DD40090094C7406F0800690094C7401F0EFB4FD
:105DE4000904C2C3803690094CE0B4031C90081B1C
:105DF40074FFF5F01249F045F0600ED2C4D2C5D25A
:105E0400C2C2C3E490094CF0FF90094CE06008C2A0
:105E1400C5D2C4C2C38005C2C3025D1420C7FD90AD
:055E2400081DE0F584FB
:015E29002256
:105E2A0090082AEFF0A3ECF0A3EDF0A3EBF0A3EABD
:045E3A00F0A3E9F0F8
:105E3E009008327403F0A374E8F0A3E584F0E4F55F
:105E4E008420C7FDD2C2C2C4D2C5E4FF90094CF073
:105E5E0030C3FDAEC1EE124C515E8C005E8F085EFB
:105E6E008F105EBA185EC5205ECD285EE8305EF0FB
:105E7E00385EF8405F08505F3A5800005E8C025F53
:105E8E0040C2C5EF700F90082AE025E044A0F5C28D
:105E9E007F03025F46EF64016003025F4690082AAB
:105EAE00E025E044A1F5C27F04025F4690082BE096
:105EBE00F5C27F05025F4690094C7403F08079EFBE
:105ECE00B4050B90082BA3E0F5C27F06806AEFB4F1
:105EDE000606D2C57F018060801890094C7404F0CC
:105EEE00805690094C7406F0804EEFB404047F0285
:105EFE00804690094C7405F0803E90082DE0FBA37F
:105F0E00E475F001124A06A9F0FAE5C2124955905D
:105F1E000831E024FFF0900830E034FFF0E070022A
:105F2E00A3E07004C2C280107F02800CD2C47F092D
:105F3E00800690094C7401F0EFB40904C2C3803698
:105F4E0090094CE0B4031C90083274FFF5F012492E
:105F5E00F045F0600ED2C4D2C5D2C2C2C3E49009DD
:105F6E004CF0FF90094CE06008C2C5D2C4C2C38099
:0F5F7E0005C2C3025E5E20C7FD900834E0F584C3
:015F8D0022F1
:10670000900853EFF0900856EBF0A3EAF0A3E9F0FD
:08671000900854ECF0A3EDF039
:10671800750F00543FF510543F605CC374409510EA
:10672800FFE4950FFE900859E0FCA3E0FDC39FEC41
:106738009E50068C0D8D0E80048E0D8F0E125CBA45
:1067480090094CE060037F0222900855E0250EF086
:10675800900854E0350DF090085BE0700B900857F6
:10676800E50D850EF01249F0C390085AE0950EF039
:10677800900859E0950DF0900859E0F50DA3E0F563
:106788000ED3E50E9400E50D94004070E50E94409C
:10679800E50D94005013125CBA90094CE060037F39
:1067A8000222E4F50DF50E80D8900853E0FFA3E02F
:1067B800FCA3E0FDA3E0FBA3E0FAA3E0F99008182E
:1067C800E4F07440125CD690094CE060037F02222A
:1067D80074C0250EF50E74FF350DF50D900855E0C3
:1067E8002440F0900854E03400F090085BE0709189
:0E67F80090085775F0401249F00267897F0043
:01680600226F
:1087B400900830E4F0A304F0125E2A90094CE060C3
:0787C400037F01227F002268
:10874F0090094BEBF07B017A09794B900859E4F0D3
:0A875F00A304F0E4A3F01267002267
:1085E000C00790086BE0FFA3E0900830CFF0A3EF46
:1085F000F0D007125E2A90094CE060037F01227FD1
:02860000002256
:10876900C007900873E0FFA3E0900859CFF0A3EF8A
:0A877900F0E4A3F0D007126700221D
:06892D00140A05140A05FE
:0F6DEF004107640048073C00000000000000005E
:06833200E0FF7B027D026A
:1083380090094DEBF0900764E070159008AB04F0DD
:10834800A37407F0A37444F090094DE0FB027F2862
:0F83580090094DE0FF7B017A077944127A3222B7
:05710A0090094EEFF0BA
:10710F007F20900744E4F0A3DFFC900748E4F0A34E
:10711F0004F090094E128332E490074CF0A3F0A3D1
:10712F00E4F0900704E0FE90074EE04EF0A3E0F08D
:10713F00E054CFF04410F0900705E07E00C4F854FF
:10714F000FC868FFEEC454F048FE900750E04EFEA3
:10715F00A3E04FFF900750EEF0FCA3EFF0FD900778
:10716F0006E0FFECFEED4FFF900750EEF0A3EFF0BF
:10717F0090094EE0FF7B067D041283387F027E006C
:10718F0012824C90094EE0FF7B0FE4FD1283030047
:01719F0022CD
:078906007F557E0002824C48
:107E8F00900921EDF0A3EBF0900920EFF07B0FE4C8
:107E9F00FD128303900922E09007486009E04440F7
:107EAF00F0A3E0F08004E054BFF090074FE054F0EF
:107EBF00F0900921E0540FFF90074EE0F0A3E04F40
:0D7ECF00F0900920E0FF7B057D0202833862
:10880D00EF9007486008E04420F0A3E0F022E05428
:03881D00DFF02267
:0D6F23009008CEECF0A3EDF09008CDEFF05B
:106F30007B0FE4FD1283039008CEE07002A3E070A3
:106F40000A9008CE7422F0A3742EF09008CEE0FED2
:106F5000A3E0FFC394B0EE941D40091272B99008EB
:106F6000D0EE80099008CEE0FFA3E0A3CFF0A3EF1E
:106F7000F09008D0E04480FFA3E090074ACFF0A350
:106F8000EFF09008CDE0FF7B037D0312833890087B
:106F9000CD1282FD900758E030E6F390074AE054A6
:106FA0007FF09008CDE0FF7B037D031283389008CB
:106FB000CD1282FD900758E0A320E6F29008CDE0C4
:086FC000FF7B0B7D0B02830334
:0E77300090090DE0FF900003124A1CFDACF022
:0B773E00900923EFF0A3ECF0A3EDF0A6
:10774900EF25E0243CF582E43407F583E0FEA3E06D
:107759006D7002EE6C6043900923E0FFA3E0FCA387
:10776900E0FD126F23900923E025E0243CF582E433
:107779003407F583E0FEA3E04E70031282C090093E
:1077890024E0FEA3E0FF900923E025E0243CF582F4
:0A779900E43407F583EEF0A3EFF0EF
:0177A30022C3
:107A9B00900704E0FE90074EE04EF0A3E0F0900755
:107AAB0005E07E00C4F8540FC868FFEEC454F048DC
:107ABB00FE900750E04EFEA3E04FFF900750EEF014
:107ACB00FCA3EFF0FD900706E0FFECFEED4FFF90FF
:107ADB000750EEF0A3EFF0E490094FF090094FE060
:107AEB00FFD39403500F7B067D0512833890094F0B
:057AFB00E004F080E74B
:017B00002262
:107CEC00900950EFF0ED9007486009E04402F0A3D2
:107CFC00E0F08004E054FDF0900748E04401F0A36C
:107D0C00E0F09009501283321282FA900758E0305A
:107D1C00E6F6900748E054FEF090095012833212B8
:107D2C0082FA900758E0A320E6F5900950E0FF7B1B
:097D3C000B7D0B1283037F002272
:1087CB007B0B7D0BE4FF12830390075AE05403FEEF
:0787DB00A3E0FF12788522E4
:07890D00900758A3E0FF22D0
:0988F500900758A3E0FF7E002269
:088212009008F9EEF0A3EFF073
:10821A00E4A3F0A3F09008F9E0FEA3E0FFC39008FE
:10822A00FCE09F9008FBE09E50177FF47E011286C7
:10823A00849008FCE004F070DC9008FBE004F08015
:01824A00D45F
:01824B002210
:0872B900900893EEF0A3EFF042
:1072C10078957C087D017BFF7A89792D7E007F038B
:1072D10012489490074EA3E0FD5430FFE4C4F854E3
:1072E100F0C8EFC4540F48FBED54C09008987009E2
:1072F1007422F0A3742EF08007741DF0A374B0F013
:10730100900898E0FEA3E0FFC3900894E09F9008E6
:1073110093E09E5008900893EEF0A3EFF090089848
:10732100E0FEA3E0FFC3900894E09FFF900893E084
:107331009EFE74952BF582E43408F583E0FD7C0014
:0373410012499B53
:017344002226
:04868400AD07AC068C
:108688007B01EDAE047805CEC313CE13D8F9FFEB0A
:09869800D39FE49E50030B80E91E
:0186A10022B6
:08824C009008FDEEF0A3EFF035
:10825400E4A3F0A3F09008FDE0FEA3E0FFC39009BF
:1082640000E09F9008FFE09E50177FE87E03128293
:1082740012900900E004F070DC9008FFE004F08044
:01828400D425
:0182850022D6
:0982FA00900950E0FF7B0A7D0AA7
:10830300900951EBF0900764E070159008A404F015
:10831300A37407F0A37444F0900951E0FB027EDCE0
:0F832300900951E0FF7B017A07794412764222DC
:10815C00900952E584F075840F43A640D2A5C2A0C5
:10816C00C2A1C2A2C2A3C2A6C2A47F647E00128214
:10817C0012D2A47F647E00128212D2A0D2A1D2A20B
:0D818C00D2A353A6BFD2A6900952E0F584FD
:0181990022C3
:0878850090089AEEF0A3EFF069
:10788D00789C7C087D017BFF7A8979307E007F03AF
:10789D0012489490074EA3E0FD5430FFE4C4F85411
:1078AD00F0C8EFC4540F48FFED54C090089F700905
:1078BD007422F0A3742EF08007741DF0A374B0F041
:1078CD00749C2FF582E43408F583E0FF7E00900868
:1078DD009AE0FCA3E0FD1249899008A0E02FFF90EB
:0578ED00089FE03EFED3
:0178F2002273
:1082860012815CE4900953F0900953E0FFD3940304
:108296005027127D45900953E0FF12710A90095349
:1082A600E0FF7B017D0F127E8F900953E0FF125095
:0982B60036900953E004F080CF7A
:0182BF00229C
:10846D007B007A007900EF14601214601714601C01
:10847D002403701E7B017A0679A580167B017A068E
:10848D0079AA800E7B017A0679AF80067B017A0688
:02849D0079B4B0
:01849F0022BA
:05706D00900901EFF0A5
:1070720012846DA3EBF0A3EAF0A3E9F0900002748E
:10708200011249229000021248D3FF90073BE0FD13
:107092003395E0FCD3EF9DEC6480F8748098401344
:1070A200900902E0FBA3E0FAA3E0F9900002740168
:1070B200124967900902E0FBA3E0FAA3E0F990000D
:1070C200021248D325E024DAF582E43406F583E09F
:1070D200FCA3E0FD900901E0FF12773E900902E077
:1070E200FBA3E0FAA3E0F99000021248D325E024C2
:1070F200DAF582E43406F583E0FFA3E0900003CFE3
:077102008FF0124AA1D20038
:017109002263
:05734500900905EFF0C6
:10734A0012846DA3EBF0A3EAF0A3E9F0ED60047FE9
:10735A00048005900905E0FF1278F3900906E0FB26
:10736A00A3E0FAA3E0F9900002EF12496790090638
:10737A00E0FBA3E0FAA3E0F99000021248D325E06B
:10738A0024DAF582E43406F583E0FCA3E0FD9009F3
:10739A0005E0FF12773E900906E0FBA3E0FAA3E0BE
:1073AA00F99000021248D325E024DAF582E4340683
:1073BA00F583E0FFA3E0900003CF8FF0124AA1D239
:0173CA0000C2
:0173CB00229F
:0278F300AD07DF
:1078F500900939E4F0A374C6F0900939E0C313FE8A
:10790500A3E013FFED25E024A6F582E43407F58313
:10791500E0FAA3E0D39FEA9E50037F0022ED25E025
:1079250024A6F582E43407F583E0FAA3E0C394E0E6
:10793500EA940E40037F1422ED25E024A6F582E4A7
:107945003407F583E0FCA3E02FFFEC3EFE900939F8
:08795500E0FCA3E0FD12499BD8
:01795D002207
:1074D1009008C17407F0A374F8F0EF25E024A6F535
:1074E10082E43407F583E0FEA3E0FBAA06E4F9F8A1
:1074F1009008C1E0FEA3E0FFE4FCFD124ACE900833
:10750100C3124C149008C3E0FCA3E0FDA3E0FEA36A
:10751100E0FFE47B7A7A0FF9F8124B599008C31215
:107521004C149008C3E0FCA3E0FDA3E0FEA3E0241B
:107531002EFFEE3422FEE43DFDE43CFC9008C31234
:0C7541004C149008C3A3A3E0FEA3E0FFDD
:01754D00221B
:0F8867007C007D0A12499B7C007D0A1249892200
:0571A000900909EFF069
:1071A50012846DA3EBF0A3EAF0A3E9F090000112BD
:1071B50048D37035900909E0FF1278F390090AE089
:1071C500FBA3E0FAA3E0F9900002EF1249679000F3
:1071D500021248D325E024DAF582E43406F583E08B
:1071E500FFA3E0900003CF802C90090AE0FBA3E009
:1071F500FAA3E0F9900002E4124967900909E0FF5B
:107205001274D112886790090AE0FBA3E0FAA3E0A3
:10721500F9900003EE8FF0124AA190090912773315
:07722500128734D205D200EC
:01722C00223F
:056AB60090090DEFF056
:106ABB0012846DA3EBF0A3EAF0A3E9F090000112AE
:106ACB0048D3705390090EE0FBA3E0FAA3E0F990D2
:106ADB0000021248D3FFD3941440079000027414A1
:106AEB00800AEFD394009000025004E402496774CB
:106AFB00FF1249229000021248D325E024DAF582D6
:106B0B00E43406F583E0FFA3E0900003CF8FF0128F
:106B1B004AA1127730806390090EE0FBA3E0FAA341
:106B2B00E0F9900003124A1CFFAEF0C3942EEE94D2
:106B3B0022500A900003742275F02E8011D3EF942B
:106B4B0026EE942A400B900003742A75F026024A15
:106B5B00A1C3EF9438EE9422402790000374FF7585
:106B6B00F0F6124A5412773090090EE0FBA3E0FACC
:106B7B00A3E0F9900002E4124967128734D205D2E0
:016B8B000009
:016B8C0022E6
:05690000900911EFF009
:1069050012846DA3EBF0A3EAF0A3E9F09000011265
:1069150048D37056900912E0FBA3E0FAA3E0F99082
:1069250000021248D3FFC394144007900002741468
:10693500800AEFC394009000025004E40249677492
:10694500011249229000021248D325E024DAF5828B
:10695500E43406F583E0FFA3E0900003CF8FF01247
:106965004AA19009111277338065900912E0FBA3C3
:10697500E0FAA3E0F9900003124A1CFFAEF0C394BD
:106985002EEE9422500A900003742275F02E801189
:10699500C3EF9426EE942A400B900003742A75F0F9
:1069A50026024AA1D3EF941CEE942A5029900003A5
:1069B500E475F00A124A54900911127733900912BE
:1069C500E0FBA3E0FAA3E0F9900002E412496712A4
:0669D5008734D205D20058
:0169DB002299
:106DFE0045079200000000004A07970000000000BF
:106E0E0000000000004507A1FFFFFFFFFF4A07A695
:106E1E000000000000000000000041078CE845075C
:066E2E008D0000000000D1
:105B410090078CE0603BE4900954F0900954E0FF29
:105B510025E0247DF582E43408F583E0FCA3E0FD33
:105B6100EF25E02481F582E43408F583ECF0A3ED20
:105B7100F0900954E004F0E0B402D090078CE014F6
:105B8100F090078CE070047D0180027D00E4FF123B
:105B910056F390078CE070047D0180027D007F0147
:105BA1001256F3E4900954F0900954E0FFD39404A1
:105BB1004003025CB9EF25E02497F582E43407F550
:105BC10083E0FEA3E0FFD39496EE94004031900968
:105BD10054E024A1F582E43407F583E0D3940F5017
:105BE10003025C7C900954E0FD2492F582E43407C1
:105BF100F5837403F074A12DF582E4340780789065
:105C01000954E02492F582E43407F583E0FDB403FE
:105C11003C900954E0FC248DF582E43407F583E0DF
:105C210004F0748D2CF582E43407F583E0D3940FEE
:105C31004049900954E0FC2492F582E43407F5834D
:105C41007401F0748D2CF582E43407802AEDB401DF
:105C510012900954E02492F582E43407F58374022A
:105C6100F08018C3EF9430EE9400500F900954E087
:105C71002492F582E43407F583E4F0900954E0FFBF
:105C810025E02497F582E43407F583E4F0A3F0746A
:105C9100A12FF582E43407F583E0C39414501090EA
:105CA1000954E024A1F582E43407F583E004F0907F
:085CB1000954E004F0025BA9B4
:015CB90022C8
:1084F900AE84E4F5848FBBFF0FEFB40AFBC2EDD263
:10850900EC30EDFD90093BE5BFF0A3E5BEF0AF0609
:0A8519008F8490093BE0FEA3E0FF11
:018523002235
:10811B00AE84ADE775840253E7FBE5E85401FC8FB1
:10812B00BBE4FF0FEFB40AFBC2EDD2EC30EDFDE484
:10813B0090093DF0A3E5BEF053E8FEAF04EC42E836
:10814B00AF058FE7AF068F8490093DE0FEA3E0FFFC
:01815B002201
:05879C00E0FCA3E0FD7C
:1087A100D3EF9DEC6480F8EE648098400122AE0422
:0387B100AF0522EF
:0350060002624AF9
:10624A00C0E0C0F0C083C082C0D075D000C000C01A
:0D625A0001C002C003C004C005C006C0079B
:106267009008D2E4F09008D2E0FFD39404400302F0
:0262770062FEC5
:106279001284F9E4FCFDC004C005C006C0079008FB
:10628900D2E025E024A6F582E43407F583E0FEA3F5
:10629900E0FFE47B0FFAF9F8124ACED003D002D01E
:1062A90001D000EF2BFFEE3AFEED39FDEC38FC9002
:1062B90008D3124C149008D3E0FCA3E0FDA3E0FE40
:1062C900A3E0FF7804124C019008D3124C149008F3
:1062D900D3A3A3E0FEA3E0FF9008D2E025E024A623
:0C62E900F582E43407F583EEF0A3EFF03B
:1062F5009008D2E004F002626C7F0712811B9007C0
:106305009712879C900797EEF0A3EFF07F06128116
:106315001B90079912879C900799EEF0A3EFF07FE9
:106325000512811B90079B12879C90079BEEF0A39B
:10633500EFF07F0412811B90079D12879C90079DAB
:10634500EEF0A3EFF07F051284F9EF7804CEA2E713
:1063550013CE13D8F8FF90079F12879C90079FEEE6
:10636500F0A3EFF07F061284F990087DEEF0A3EF1D
:0E637500F07F071284F990087FEEF0A3EFF09E
:10638300D007D006D005D004D003D002D001D0006E
:0B639300D0D0D082D083D0F0D0E03218
:066E3400C10C41073B15F3
:10836700E4FFFE7D15ED25E02407F582E43407F5EB
:1083770083E0FAA3E0FB4A6016AE02AF03ED25E007
:108387002407F582E43407F583E4F0A3F080050DB4
:04839700EDB41AD156
:01839B0022BF
:1064CD009008C7EEF0A3EFF0A3EDF0A3EBF0A3EA75
:0464DD00F0A3E9F04F
:1064E1007EFFE4FCFD9008CAE0FBA3E0FAA3E0F91B
:1064F1008D827583001248D3FFC39E5004AE07AC52
:10650100050DEDB41ADFAF069008C9E0C39F500333
:106511000265EEEC25E02407F582E43407F583E01B
:10652100FEA3E0D39400EE94004072AD04EDC39459
:10653100195046ED25E02409F582E43407F583E09E
:10654100FEA3E0FFED25E02407F582E43407F5839F
:10655100EEF0A3EFF0ED2401FFE433FE9008CAE072
:10656100FBA3E0FAA3E0F98F828E831248D38D82D8
:106571007583001249670D80B4ED25E02407F5828B
:10658100E43407F583E4F0A3F09008CAE0FBA3E04C
:10659100FAA3E0F98D82758300E4124967AF04AD77
:1065A10007EDC3941A5046ED25E02407F582E43443
:1065B10007F583E0FEA3E04E70309008C7E0FEA32C
:1065C100E0FFED25E02407F582E43407F583EEF0E2
:1065D100A3EFF09008C9E0FFA3E0FBA3E0FAA3E07A
:0D65E100F98D82758300EF0249670D80B4CB
:0165EE00228A
:10639E00D20C126C5AE49007CAF09007CAE0FFC301
:1063AE00941A502474B02FF582E43407F583E4F088
:1063BE00EF25E02407F582E43407F583E4F0A3F03B
:1063CE009007CAE004F080D27D2E7C22E4FF127783
:1063DE003E1287CB9007CFEE80389007CCE0704FFF
:1063EE00A3E0FEA3E0FFC39007D0E09F9007CFE0AD
:1063FE009E503C12890DAD079007CDE0FEA3E0FF45
:10640E007B017A0779B01264CD9007CDE0FFA3E04F
:10641E00A3CFF0A3EFF07D01E4FF127CEC9007CC4C
:10642E00EFF01287CB9007CDEEF0A3EFF080AB909C
:10643E0007CA7401F09007CAE0FF25E02405F58233
:10644E00E43407F583E0FCA3E0FDEF25E024DAF564
:10645E0082E43406F583ECF0A3EDF09007CAE00475
:10646E00F0E0B416D09006DCE0FFA3E09006DACFA1
:10647E00F0A3EFF0C20CE49007CBF09007CBE0FF57
:05648E00D3940350341B
:1064930012846D9007D1EBF0A3EAF0A3E9F090002A
:1064A300021248D325E024DAF582E43406F583E0CA
:0C64B300FFA3E0900003CF8FF0124AA17D
:0E64BF009007CBE004F080C21282C0026C5A3B
:1082C0007D14EDFF3395E0FEEF25E0FFEE33FE7405
:1082D000DA2FF58274063EF583E0FEA3E0FF4E60E0
:0182E0000F8E
:0F82E10090093FEEF0A3EFF090073BEDF0FF2286
:0982F000DDD0E490073BF0E0FF53
:0182F9002262
:0E887600E4FFFE0FBF00010EEF64054E70F52B
:0188840022D1
:1088330020F907E59A30E7F880F98F9B30FFFDC2F6
:02884300FF2212
:02843900AC078E
:10843B00AB84E4F5840CC290128876EDC4540FFF24
:10844B00AE04EEC454F04FFF128833AF05EFC454A3
:10845B00F0FF128833128876D290128876AF038F92
:01846B00848C
:01846C0022ED
:026FC800AA0716
:106FCA0074242AF582E43405F583E0FF600122EA9D
:106FDA00C39419501FEAFF7E007C007DB4124989D0
:106FEA007D1912499B900941EEF0A3EFF0C374FF9B
:106FFA009FFB8061EAC39433501FEAFF7E007C0046
:10700A007D181249897D1A12499B900941EEF0A315
:10701A00EFF0C374629FFB803CEAC3947FEA501E80
:10702A00FF7E007C007D1D1249897D4C12499B9090
:10703A000941EEF0A3EFF0C374479FFB801775F088
:10704A0003A4FFE5F0C4F854F0C8EFC4540F48FF96
:10705A00C374309FFB74242AF582E43405F583EB6C
:02706A00F0FF35
:01706C002201
:0E889400A907AF05126FC8AD07AF0102843906
:106E3A004407E0000000004407E403030303480793
:096E4A00D400000000000000006B
:104CA30090087DE0C4F854F0C8A3E0C4540F4890C2
:104CB3000927F090087FE0C4F854F0C8A3E0C45477
:104CC3000F48900928F0E4900926F0900926E0FFA8
:104CD30024E0F582E43407F583E0FE74922FF58235
:104CE300E43407F583E0B4012E900926E024E4F5CB
:104CF30082E43407F583E4F074E02FF582E43407AB
:104D0300F5837401F0EF25E024D4F582E43407F54C
:104D130083E4F0A3F0D205900926E0FF24E4F582B2
:104D2300E43407F583E06003024E0574E02FF58257
:104D3300E43407F583E0C394FF4003024DEC90098C
:104D430027E0FFFD7C009007DCECF0A3EDF0900979
:104D530026E0F925E024D4F582E43407F583E475ED
:104D6300F001124A06FAC3E5F09DEA9C5003024F94
:104D730046EFD3943C400F74E029F582E43407F501
:104D830083E004F0805F900927E0D3941E402074F1
:104D9300E029F582E43407F583E0D394FD501074E1
:104DA300E029F582E43407F583E02402F0803690AD
:104DB3000927E0D3941E502074E029F582E43407D8
:104DC300F583E0D394FB501074E029F582E43407B3
:104DD300F583E02404F0800D74E029F582E43407C0
:104DE300F58374FFF0E9024F239006BDE090092696
:104DF3006041E024E4F582E43407F5837402F002B1
:104E03004F46900926E0FF24E4F582E43407F58356
:104E1300E0FDB4022E74922FF582E43407F583E0AB
:104E230064027003024F46900796E06003024F4608
:104E3300900926E024E4F582E43407F5837401F055
:104E4300024F46ED64016003024F46900928E0FFDC
:104E5300C394FE4003024F46900926E0FD24E0F58B
:104E630082E43407F583E0D394005003024F34EF18
:104E7300FB7A009007DEEAF0A3EBF0ED25E024D403
:104E8300F582E43407F583E475F001124A06FCC3A6
:104E9300E5F09BEC9A5003024F46900927E0FFD3BD
:104EA300943C4012900926E024E0F582E43407F5AF
:104EB30083E014F08066EFD3941E4024900926E02B
:104EC300FF24E0F582E43407F583E0C39402401045
:104ED30074E02FF582E43407F583E024FEF0803C90
:104EE300900927E0D3941E5024900926E0FF24E084
:104EF300F582E43407F583E0C39404401074E02F93
:104F0300F582E43407F583E024FCF0800F90092652
:104F1300E024E0F582E43407F583E4F0900926E029
:104F230025E024D4F582E43407F583E4F0A3F0808C
:104F330012900926E024E4F582E43407F583740330
:104F4300F0D205900926E024E0F582E43407F583E6
:104F5300E0FD6E6008900926E0FF12889490092610
:0C4F6300E004F0E0D394035003024CCEB5
:014F6F00221F
:1086DE007F80900624E4F0A3DFFC7B017A067924E8
:0C86EE008B0A8A0B890C8A088909D2B516
:0186FA00225D
:1086FB00E50A850B83850C826401700AE5096582A6
:0D870B007004E50865837002FF227F0122E3
:107F7400E50A850B83850C826401700AE509658234
:107F84007004E50865837003FF802FAB0A050CE5D8
:107F94000CAA0B7002050B14F91248BAFF74019075
:107FA40006A46B700AE50C65827004E50B658370AA
:0A7FB40009750A01750B06750C240F
:017FBE0022A0
:03500300027D9D8E
:107D9D00C0E0C083C082C0D075D000C004C006C092
:017DAD0007CE
:107DAE00AF8475840FE5B0541FFE0509E509AC08D4
:107DBE007002050814F5828C83EEF0C3E50994A4D5
:107DCE00E50894064006750806750924C2B5308686
:057DDE00FDD2B58F8409
:0F7DE300D007D006D004D0D0D082D083D0E032E9
:0573CC00900915EFF02F
:1073D10012846D900916EBF0A3EAF0A3E9F0900096
:1073E100011248D3F490000112496790000112483C
:1073F100D37055900916E0FBA3E0FAA3E0F99000E1
:10740100021248D3FF604125E024DAF582E4340614
:10741100F583E0FCA3E0FD900915E0FF12773E90B3
:107421000916E0FBA3E0FAA3E0F99000021248D3A9
:1074310025E024DAF582E43406F583E0FFA3E09049
:0F7441000003CF8FF0124AA1128734D205D20078
:017450002219
:1087E20012846D7401124900B40304E41249551253
:0687F2008734D205D2001D
:0187F800225E
:107B0100E4FFFE75840F438C670FBF00010EBE0BAF
:107B1100F8BFB8F5E58C30E7FB43890453A1DFE4F6
:107B2100F58475B73075840F43A120438901758DA4
:107B310001758F01758E04FEFF0FBF00010EEF640A
:107B41000F4E70F5438902E58920E4130FBF000150
:107B51000EBE0FF3BFFFF0E4F58443EF1080E8752C
:057B61009702E4F58A23
:017B660022FC
:10857300AF8475840F75E10343E20443E3C075A43C
:108583000F7580F075A50775AD0775A6FF75A0FF7C
:0585930075A7E08F84D4
:0185980022C0
:0D88A200AF84E4F58475D48475D1038F8410
:0188AF0022A6
:10882000AF84E4F584759D0143F809759A40D2F848
:028830008F8433
:018832002223
:0F888500E4F584758810758902F584758E0222DA
:1087F900AF8475840275C90875CBB0E4F5CA75C82C
:03880900048F8455
:01880C002249
:10864400AF84E4F584F5BA75BC9875E88075840246
:10865400F5BA75BCF975E88075C4AF75C6FF8F842B
:0186640022F3
:10885600AF8443E704D2A8D2A9E4F584D2888F84F2
:0188660022EF
:1086A200127B011285731288201288A21286DE12B2
:0E86B20086441288851287F9127815028856C0
:0489440075EF102299
:1086C000C2A57F027E00128684C2A67F037E0012AE
:0E86D0008684D2A57F037E00128684D2A62265
:0576BB00900943EFF00F
:1076C0007F037E00128684C2A67F037E001286841A
:1076D000C2A59009447407F0C2A57F037E001286FC
:1076E00084900944E0FF900943E0FEA80708800267
:1076F000C313D8FC1392A67F037E00128684D2A502
:107700007F037E00128684900944E014F0E0C36495
:1077100080948050C3C2A5D2A67F027E00128684C8
:0F772000D2A57F037E0012868430A6031289440F
:01772F002237
:057C2B00900945EFF097
:107C3000A37407F0C2A57F037E00128684900946D4
:107C4000E0FF900945E0FEA807088002C313D8FCB6
:107C50001392A67F027E00128684D2A57F037E0047
:107C6000128684900946E014F0E0C364809480504A
:107C7000C3C2A5D2A67F027E00128684D2A57F034E
:0B7C80007E0012868430A603128944A7
:017C8B0022D6
:05795E00900929EFF083
:10796300E490092BF090092A7407F0C2A5D2A67FF0
:10797300037E001286847F027E00128684D2A57F56
:10798300037E0012868490092BE025E0FFA2A6E483
:10799300334FF090092AE014F0E0C36480948050E0
:1079A300CAC2A5900929E07004D2A68002C2A67FAC
:1079B300027E00128684D2A57F037E001286849005
:0479C300092BE0FFAD
:0179C700229D
:0E7A32009008D7EFF0A3EBF0A3EAF0A3E9F081
:107A4000A37402F07F201276BB9008D8E0FBA3E07D
:107A5000FAA3E0F9A3E075F002A4F58285F08312A1
:107A60004A1CE5F0FF127C2B9008D8E0FBA3E0FA5B
:107A7000A3E0F9A3E075F002A4F58285F083124A31
:107A80001CFF127C2B9008DBE004540FFFF09008E1
:0B7A9000D7E004540FB507B10286C018
:0E764200900875EFF0A3EBF0A3EAF0A3E9F0D7
:09765000A3740AF07F211276BB3D
:107659007F0112795E90087AE4F0A3EFF09008793F
:10766900E0FF900875E0C39FFF12795E90087CEFF8
:10767900F0FD90087BE0FE7C00E42DFFEC3EFE90DF
:107689000876E0FBA3E0FAA3E0F9A3E0FD75F002B8
:10769900A4F58285F083EE8FF0124AA1ED04540F10
:0576A900FF900879F0DC
:0D76AE00900875E004540FB507A10286C0D6
:0D88BD00A2B7300D01B350030080F500227A
:107E410053A6BFD2A690092C740FF0C2A57F197E4C
:107E510000128684D2A57F197E0012868490092E95
:107E6100E025E0FF90092DE033FEA2A6E433FDEF0B
:107E71004DFFEEF0A3EFF090092CE014F0E0C364A5
:0D7E810080948050C690092DE0FEA3E0FF24
:017E8E0022D1
:087FBF0090092FEEF0A3EFF092
:107FC700ED14A3F0900931E0FFC364809480403042
:107FD700C2A590092FE0FEA3E0A807088005CEC33D
:107FE70013CE13D8F91392A67F197E00128684D276
:107FF700A57F197E00128684900931E014F080C4B1
:018007002256
:0B68070090083FEFF0A3EDF0A3EBF0D2
:10681200900847E584F0A3E5E1F075840F43A640B4
:10682200900840E0B40106A3E024E080069008410D
:10683200E024C0FEE433900845F0A3CEF090083F78
:10684200E0FF7002C2A0EFB40102C2A1EFB40202E3
:10685200C2A2EFB40302C2A3900845E0FEA3E0FF88
:106862007D09127FBF900840E0B40121127E419061
:106872000842E0FBA3E0FAA3E0F9900841E075F0DA
:1068820002A4F58285F083EE8FF0124AA1900840AF
:10689200E07023900842E0FBA3E0FAA3E0F990083D
:1068A20041E075F002A4F58285F083124A1CFFAE26
:1068B200F07D10127FBFC2A57F057E0012868490F4
:1068C200083FE0FF7002D2A0EFB40102D2A1EFB400
:1068D2000202D2A2EFB40302D2A37F147E00128678
:1068E20084D2A57F197E00128684C2A553A6BFD288
:0D68F200A6900848E0F5E1900847E0F58425
:0168FF002276
:0A7EDC009008A1EFF09008A3EBF06E
:107EE6009008A7EDF0EB04540F9008A3F09008A1BA
:107EF600E0FF9008A4E0F9A3E0FAA3E0900842C9E5
:107F0600F0A3EAF0A3E9F09008A7E0FB7D01126870
:107F1600079008A7E004540FFFF09008A3E0B50708
:017F2600CC8E
:017F27002237
:0A7F28009008A8EFF09008AAEBF013
:107F32009008AEEDF0EB04540F9008AAF09008A858
:107F4200E0FF9008ABE0F9A3E0FAA3E0900842C991
:107F5200F0A3EAF0A3E9F09008AEE0FBE4FD1268BA
:107F6200079008AEE004540FFFF09008AAE0B507AE
:017F7200CC42
:017F730022EB
:0E6E530044087D00000000440881000000009B
:0856F3009007E8EFF0A3EDF0D1
:1056FB00E4A3F0A3F09007E8E0FD25E02481F58218
:10570B00E43408F583E0FEA3E0FFED25E0247DF50E
:10571B0082E43408F583E0FCA3E0C39FFDEC9EFC20
:10572B00C3ED9440EC6480948040089007EAE4F069
:10573B00A304F0D3ED94C0EC6480947F500874FF05
:10574B009007EAF0A3F09007EAE0FCA3E0FD4C70B1
:0F575B0003025975EDF47002ECF4600302583349
:10576A00FCFD9007F4124C14E47F01FEFDFC900747
:10577A00F4E0F8A3E0F9A3E0FAA3E0FBC3124BEBD1
:10578A00500A9007F4124C20000000019007E8E04C
:10579A0025E024B9F582E43406F583E0FEA3E0FFB0
:1057AA00E4FCFD7BFF7A0FF9F8124ACE9007F4E089
:1057BA00F8A3E0F9A3E0FAA3E0FB1280D79007EC84
:1057CA00124C149007E8E025E0247DF582E43408C1
:1057DA00F583E0FEA3E0FFE4FCFD9007ECE0F8A30C
:1057EA00E0F9A3E0FAA3E0FB124ACE9007F0124CCC
:1057FA0014E47BFF7A0FF9F89007F0E0FCA3E0FDD0
:10580A00A3E0FEA3E0FF1280D79007E8E025E0249A
:10581A00B9F582E43406F583EEF0A3EFF09007E9D8
:06582A00E0700302594F7B
:1058300002594C9007EAE07004A3E064016003029F
:02584000594FBE
:105842009007E8E025E024B9F582E43406F583E028
:10585200FEA3E0FBC374FF9BFF740F9EFEE4940063
:10586200FDE49400FCE47BFF7A0FF9F8124ACE9033
:1058720007EC124C149007E8E025E02481F582E45D
:105882003408F583E0FEA3E0FBC374FF9BFF740FB3
:105892009EFEE49400FDE49400FC9007F0124C1488
:1058A200E47F01FEFDFC9007F0E0F8A3E0F9A3E03D
:1058B200FAA3E0FBC3124BEB500A9007F0124C2004
:1058C200000000019007ECE0FCA3E0FDA3E0FEA3D2
:1058D200E0FFA3E0F8A3E0F9A3E0FAA3E0FB128063
:1058E200D79007EC124C149007E8E025E0247DF5F0
:1058F20082E43408F583E0FEA3E0FBC374FF9BFF60
:10590200740F9EFEE49400FDE49400FC9007ECE02A
:10591200F8A3E0F9A3E0FAA3E0FB124ACEE47BFF8E
:105922007A0FF9F81280D7C374FF9FFF740F9EFE9F
:105932009007E8E025E024B9F582E43406F583EE29
:0D594200F0A3EFF09007E9E0600312873456
:10594F009007E8E0FF25E0247DF582E43408F58335
:10595F00E0FCA3E0FDEF25E02481F582E43408F5B7
:06596F0083ECF0A3EDF053
:01597500220F
:0D6E61004A07F87E306D79335B5F707F7BF0
:1060EE00900955E584F01288E0C291E4FD7C03909E
:1060FE000802E4F0A3DCFC7C007D032004033003E3
:10610E0007900804E04401F09006BDE06007900897
:10611E0004E04402F09006A5E0FFB40109900804E3
:10612E00E04404F0800BEFB40207900804E044084A
:10613E00F09006A6E09008047006E04410F080048B
:10614E00E04420F0E4FF74E02FF582E43407F58399
:10615E00E06015900803E0FE7401A807088002C3F2
:10616E0033D8FC4E900803F00FEFB404D99006AB71
:10617E00E09008037006E04420F08004E04410F044
:10618E009006AAE0FFB40109900803E04480F08075
:10619E000BEFB40207900803E04440F09006B5E020
:1061AE009008027006E04402F08004E04401F09092
:1061BE0006B4E0FFB40109900802E04408F0800B39
:1061CE00EFB40207900802E04404F09006B0E090AD
:1061DE0008027006E04420F08004E04410F09006BF
:1061EE00AFE0FFB40109900802E04480F0800BEFAD
:1061FE00B40207900802E04440F053E7FBE4F58454
:10620E00FCFD53F87FE59A20E7FB74022DF58274AE
:10621E00083CF583E0F59BE4FFFE0FBF00010EEF97
:10622E0064144E70F50DBD00010CED64034C70D27C
:0B623E00D29143E704900955E0F5847D
:016249002232
:0A88E0007F03900802E4F0A3DFFC20
:0188EA00226B
:057B6700900932EFF06F
:107B6C00E4F9A3F0A3F0900933E0FEA3E0FFC39483
:107B7C0008EE64809480504374017E00A80708804E
:107B8C0005C333CE33CED8F9FF900932E0FDE4FEC5
:107B9C00EF5DFFA3A3E0FDC374079DFDEFA80508EF
:107BAC008005C333CE33CED8F949F9900934E004BB
:0D7BBC00F070B3900933E004F080ABAF012E
:017BC9002299
:06754E007D047F027E00B7
:107554009008DCEEF0A3EFF0A3EDF0A3EAF0A3EBC8
:01756400F036
:10756500AF84E4F58453E7FBC292FEEEFD9008DCA0
:10757500E07003A3E06D702553F87FE59A20E7FBE3
:107585009008DEE0F59BE4F909E9B414FB9008DF07
:10759500A3E0F59BE4F909E9B414FB801A53F87FDD
:1075A500E59A20E7FBE4F59BF909E9B414FBE4F55A
:1075B5009BF909E9B414FB0EEEB403AFD29243E78D
:0375C500048F84AC
:0175C80022A0
:1077A4007B1F7A007D051275507B3E7D0612755055
:1077B4007B4E7D011275507B377D021275507B0E16
:1077C4007D031275507B7712754E9007FAE0FB7DAE
:1077D400017F017E001275549007FFE0FB7D027F5C
:1077E400017E001275549007FAE0FB7D037F017E51
:1077F400001275547B4F7D047F017E001275547C0A
:1078040001AD04E4FBFAFFFE1275540CECB409F16B
:017814002251
:10781500E4900956F0900956E0FFC3940350467E64
:1078250000E4FBFA7D0F127554900956E0FF7E00C7
:107835000B7D0C127554900956E0FF7E001B7D09E7
:10784500127554900956E0FF7E007D0A127554901A
:107855000956E0FF7E007B077D0B12755490095693
:10786500E004F080B0E4900956F0900956E0FFD3AB
:0F7875009403500B127D45900956E004F080EB10
:0178840022E1
:106C5A00300C6F7B5B7A007D011275507B4E7D0292
:106C6A001275507B777D031275501B12754EE4FB2B
:106C7A007D057F02FE127554E47D067F02FE1275C1
:106C8A00549009577401F0900957E0FDD3940450C9
:106C9A0011E4FBFA7F01FE127554900957E004F0E3
:106CAA0080E59009577401F0900957E0FDD39408E4
:106CBA00505AE4FBFAFFFE127554900957E004F0AB
:106CCA0080E630012D7B4F7A007D011275507B3DA5
:106CDA007D021275507B067D031275507B0F12756B
:106CEA004E7B5B7D051275507B677D0612755002DF
:106CFA00546FE4900957F0900957E0FFD39403507A
:0C6D0A000B125036900957E004F080EBAB
:016D1600225A
:10546F00900704E0FF7E00900947EEF0A3EFF07C79
:10547F00007D0A12499B74F82DF58274073CF58361
:10548F00E0FB7A007D047F017E001275549009477E
:10549F00E0FEA3E0FF7C007D0A12499B900947EED6
:1054AF00F0A3EFF07C007D0A12499B74F82DF58272
:1054BF0074073CF583E0FB7D037F017E001275547A
:1054CF00900947E0FEA3E0FF7C007D0A12499B9004
:1054DF000947EEF0A3EFF07C007D0A12499B74F8A8
:1054EF002DF58274073CF583E0FB7D027F017E0082
:1054FF00127554900947E0FEA3E0FF7C007D0A126D
:10550F00499B900947EEF0A3EFF04E7008FB7D0129
:10551F007F01FE8023900947E0FEA3E0FF7C007D22
:10552F000A12499B74F82DF58274073CF583E0FB52
:10553F007A007D017F017E00127554900705E0FF10
:10554F007E00900947EEF0A3EFF07C007D0A124930
:10555F009B74F82DF58274073CF583E0FB7A007D90
:10556F0004E4FFFE127554900947E0FEA3E0FF7CB0
:10557F00007D0A12499B900947EEF0A3EFF07C00E3
:10558F007D0A12499B74F82DF58274073CF583E070
:10559F00FB7D03E4FFFE127554900947E0FEA3E084
:1055AF00FF7C007D0A12499B900947EEF0A3EFF0B4
:1055BF007C007D0A12499B74F82DF58274073CF527
:1055CF0083E0FB7D02E4FFFE127554900947E0FE75
:1055DF00A3E0FF7C007D0A12499B900947EEF0A3E0
:1055EF00EFF04E7005FB7D018020900947E0FEA390
:1055FF00E0FF7C007D0A12499B74F82DF582740739
:10560F003CF583E0FB7A007D01E4FFFE12755490B8
:10561F000706E0FF7E00900947EEF0A3EFF07C0055
:10562F007D0A12499B74F82DF58274073CF583E0CF
:10563F00FB7A007D08E4FFFE127554900947E0FEE7
:10564F00A3E0FF7C007D0A12499B900947EEF0A36F
:10565F00EFF07C007D0A12499B74F82DF5827407D8
:10566F003CF583E0FB7D07E4FFFE1275549009477C
:10567F00E0FEA3E0FF7C007D0A12499B900947EEF4
:10568F00F0A3EFF07C007D0A12499B74F82DF58290
:10569F0074073CF583E0FB7D06E4FFFE1275549022
:1056AF000947E0FEA3E0FF7C007D0A12499B9009A9
:1056BF0047EEF0A3EFF04E7005FB7D0580209009BB
:1056CF0047E0FEA3E0FF7C007D0A12499B74F82D92
:1056DF00F58274073CF583E0FB7A007D05E4FFFE5D
:0356EF00127554DD
:0156F2002295
:10503600EF1470030251701470030252741470035B
:105046000253712403600302546E9006A7E075F0C4
:105056000A84FF7E00900949EEF0A3EFF024F8F5EC
:1050660082E43407F583E0FB7A007D057F02127542
:10507600549006A7E075F00A84AFF07E00900949C7
:10508600EEF0A3EFF024F8F582E43407F583E0FBB5
:105096007D067F021275549006A8E0FEA3E0FF7C11
:1050A600007D0A12499B900949EEF0A3EFF07C00BF
:1050B6007D0A12499B74F82DF58274073CF583E04E
:1050C600FB12754E900949E0FEA3E0FF7C007D0AC5
:1050D60012499B900949EEF0A3EFF07C007D0A127D
:1050E600499B74F82DF58274073CF583E04480FBF8
:1050F6007D03127550900949E0FEA3E0FF7C007D18
:105106000A12499B900949EEF0A3EFF07C007D0A54
:1051160012499B74F82DF58274073CF583E0FB7DFC
:1051260002127550900949E0FEA3E0FF7C007D0A5B
:1051360012499B900949EEF0A3EFF04E7008FB7DF3
:10514600017F0202536D900949E0FEA3E0FF7C0057
:105156007D0A12499B74F82DF58274073CF583E0AD
:10516600FB7A007D017F0202526F9006ABE0700968
:10517600A3E0FF900949E480139006ADE0FEA3E0AA
:10518600FF7C007D0A12499B900949EEF0A3EFF0DF
:10519600900949E0FEA3E0FF7C007D0A12499B745A
:1051A600F82DF58274073CF583E0FB7A007D047FD9
:1051B600017E00127554900949E0FEA3E0FF7C00D1
:1051C6007D0A12499B900949EEF0A3EFF07C007D21
:1051D6000A12499B74F82DF58274073CF583E0FFAB
:1051E6009006ABE05480FDEF4DFB7D037F017E0012
:1051F600127554900949E0FEA3E0FF7C007D0A1277
:10520600499B900949EEF0A3EFF07C007D0A124914
:105216009B74F82DF58274073CF583E0FB7D027FD5
:10522600017E00127554900949E0FEA3E0FF7C0060
:105236007D0A12499B900949EEF0A3EFF04E7008E3
:10524600FB7D017F0102536D900949E0FEA3E0FF5B
:105256007C007D0A12499B74F82DF58274073CF593
:1052660083E0FB7A007D017F017E0002546B90068D
:10527600B0E07009A3E0FF900949E480139006B2FC
:10528600E0FEA3E0FF7C007D0A12499B900949EEEF
:10529600F0A3EFF0900949E0FEA3E0FF7C007D0A51
:1052A60012499B74F82DF58274073CF583E0FB7A6E
:1052B600007D04E4FFFE127554900949E0FEA3E068
:1052C600FF7C007D0A12499B900949EEF0A3EFF09E
:1052D6007C007D0A12499B74F82DF58274073CF513
:1052E60083E0FF9006B0E05480FDEF4DFB7D03E4C4
:1052F600FFFE127554900949E0FEA3E0FF7C007D95
:105306000A12499B900949EEF0A3EFF07C007D0A52
:1053160012499B74F82DF58274073CF583E0FB7DFA
:1053260002E4FFFE127554900949E0FEA3E0FF7CFB
:10533600007D0A12499B900949EEF0A3EFF04E70EA
:1053460005FB7D018020900949E0FEA3E0FF7C007B
:105356007D0A12499B74F82DF58274073CF583E0AB
:10536600FB7A007D01E4FFFE02546B9006B5E07007
:1053760009A3E0FF900949E480139006B7E0FEA375
:10538600E0FF7C007D0A12499B900949EEF0A3EFED
:10539600F0900949E0FEA3E0FF7C007D0A12499BDC
:1053A60074F82DF58274073CF583E0FB7A007D08DE
:1053B600E4FFFE127554900949E0FEA3E0FF7C006D
:1053C6007D0A12499B900949EEF0A3EFF07C007D1F
:1053D6000A12499B74F82DF58274073CF583E0FFA9
:1053E6009006B5E05480FDEF4DFB7D07E4FFFE120D
:1053F6007554900949E0FEA3E0FF7C007D0A12493E
:105406009B900949EEF0A3EFF07C007D0A12499BC0
:1054160074F82DF58274073CF583E0FB7D06E4FF06
:10542600FE127554900949E0FEA3E0FF7C007D0A58
:1054360012499B900949EEF0A3EFF04E7005FB7DF3
:10544600058020900949E0FEA3E0FF7C007D0A125A
:10545600499B74F82DF58274073CF583E0FB7A00CE
:085466007D05E4FFFE12755400
:01546E00221B
:107D4500EF14601D14602D14603C240370497C0100
:107D5500AD04E4FBFA7F02FE1275540CECB409F095
:107D6500227C01AD04E4FBFA7F01FE1275540CEC94
:107D7500B405F0227C01AD04E4FBFAFFFE12755454
:107D85000CECB405F1227C05AD04E4FBFAFFFE1210
:077D950075540CECB409F178
:017D9C0022C4
:1074510079FF7FFF7EFFE4FD7CFFFB74E02BF5826B
:10746100E43407F583E07003AF03220BEBB404EBC4
:10747100E4FB74E42BF582E43407F583E0B40114F2
:1074810074E02BF582E43407F583E0F9C39E5004E0
:10749100AF03AE010BEBB404D9EFF4600122E4FBBE
:1074A10074E42BF582E43407F583E0701474E02B67
:1074B100F582E43407F583E0FFD39C4004AD03ACCF
:0F74C100070BEBB404DAEDF46003AF05227F0094
:0174D0002299
:0B6E6E004206D70019C10E4106D900F2
:06893300E49006D9F022D9
:078914009006D97401F02266
:106E7A00E4900958F0900958E0FFD394155058EF60
:106E8A0025E024DAF582E43406F583E0FEA3E0FF88
:106E9A00C3942EEE94225018900958E025E024DA83
:106EAA00F582E43406F5837422F0A3742EF0801F71
:106EBA00D3EF9426EE942A4016900958E025E02450
:106ECA00DAF582E43406F583742AF0A37426F09086
:106EDA000958E004F0809EE4900958F0900958E0BF
:106EEA00FFD39403503212846D900003124A1CFFA0
:106EFA00AEF0C3942EEE942250028009D3EF94266A
:106F0A00EE942A400B900003742275F02E124AA1C7
:086F1A00900958E004F080C466
:016F2200224C
:1079C8009006A7E0FF9006ACE0B507179006A8E080
:1079D800FEA3E0FF9006ADEEF0FCA3EFF0FD7F0103
:1079E80012773E9006A7E0FF9006B1E0B507179022
:1079F80006A8E0FEA3E0FF9006B2EEF0FCA3EFF0CD
:107A0800FD7F0212773E9006A7E0FF9006B6E0B52C
:107A180007179006A8E0FEA3E0FF9006B7EEF0FC7B
:0A7A2800A3EFF0FD7F0312773E226A
:1081D700E4FF9007047408F0E4A3F0A3F0EF25E0B0
:1081E70024DAF582E43406F583E4F0A3F00FEFB464
:1081F70015EB7EE27FF07B017A0679DA90088AE454
:0B820700F0A3742DF012800802854DDA
:106B8D009009197402F0E4A3F0A3F0A3F01288FEAB
:106B9D007EE27FEE7B017A09791990088AE4F0A3F1
:106BAD0004F012800812854DE490091BF090091B2A
:106BBD00E0FFD39403502B12846D7401124955F5E7
:106BCD0082758300E4124967900002E412496790D0
:106BDD000003742275F02E124AA190091BE004F0F7
:106BED0080CBE49006B9F0A3F09006BDF09006BB03
:106BFD00F0A3F0D200D20590091AF090091AE0FF27
:106C0D00C3941E502A75F019EFA42400F582E5F007
:106C1D0034E0AF82FE7B017A0679A590088AE4F014
:106C2D00A37419F012800890091AE004F080CC12B8
:106C3D00854D1281D77EE27FEF7B017A09791C9019
:0D6C4D00088AE4F0A304F012800802854DCF
:10873400200E1730021030040F9006D9E070097F24
:0B8744005E1286028002D203D20E22D9
:1084A00090E2EFE493F4600990E2EEE493640260FA
:1084B00003126B8D78DA7C067D017BFF7AE279F01E
:0D84C0007E007F2D124894E49006A4F02267
:108718001288FE7EE27FF07B017A0679DA90088A79
:0C872800E4F0A3742DF012800802854DCF
:108524009006A4E0FFC3941E501CEF75F019A42418
:1085340000F974E035F0FA7BFF78A57C067D017EB6
:09854400007F19124894C20E22B6
:10839C009006A4E0C3941E502B1288FE9006A4E015
:1083AC0075F019A42400F582E5F034E0AF82FE7B71
:1083BC00017A0679A590088AE4F0A37419F012806A
:0583CC000812854D229E
:0689390012839CC20E2215
:0389480002893968
:0869DC00900806EDF0A3EBF0BA
:1069E400E490080BF0900808E004F090080CEFF035
:1069F400A3EBF0900806E0FF90080CE0FED39F4064
:106A040003026A9775F019EEA42400F582E5F034C8
:106A1400E0AF8290080EF0A3EFF090080DE075F05F
:106A240019A42400F582E5F034E0AF82900810F058
:106A3400A3EFF0E4900809F0A3F0900810E475F0D7
:106A440001124A06AFF0FE90080EE0FCA3E0F582C6
:106A54008C83E493FD12722D90080FE004F070060D
:106A640090080EE004F090080AE004F07006900824
:106A740009E004F0C390080AE09419900809E0942E
:106A84000040B712854D90080CE004F0A3E004F038
:106A94000269F79006A4E0FF900807E0D39F500C2A
:106AA400A3E0C39F400690080B7401F090080BE02C
:016AB400FFE2
:016AB50022BE
:0F59760090081FEDF090081EEFF0900820EBF066
:10598500E4A3F0900826EFF0A3EBF090081FE0FFEA
:10599500900826E0D39F4003025AF4A3E075F0195E
:1059A500A42400F582E5F034E0AF82900822F0A34C
:1059B500EFF0E4900828F0A3F0900828E0FEA3E0BB
:1059C500FFC39419EE94005038900822E0FCA3E040
:1059D500F5828C83E493FD74BE2FF582E43406F5DD
:1059E50083EDF0900823E004F07006900822E004AF
:1059F500F0900829E004F070C0900828E004F080D9
:105A0500B8900826E075F019A42400F582E5F03475
:105A1500E0AF82900824F0A3EFF0900827E075F03E
:105A250019A42400F582E5F034E0AF82900822F055
:105A3500A3EFF0E4900828F0A3F0900822E475F0B5
:105A450001124A06AFF0FE900824E0FCA3E0F582BF
:105A55008C83E493FD12722D900825E004F0700606
:105A6500900824E004F0900829E004F070069008FE
:105A750028E004F0C3900829E09419900828E094E0
:105A85000040B7900826E075F019A42400F582E5DA
:105A9500F034E0AF82900824F0A3EFF0E4900828FA
:105AA500F0A3F0900828E0FCA3E0FDC39419EC9462
:105AB50000502C900824E475F001124A06AFF0FE60
:105AC50074BE2DF582E43406F583E0FD12722D9047
:105AD5000829E004F070CC900828E004F080C41296
:105AE500854D900826E004F0A3E004F0025990905B
:105AF50006A4E0FF900820E0FED39F502090081EEA
:105B0500E0FDA3E0C39DFDE49400FCEE7A002DFDCD
:105B1500EA3CFCC3ED9F7480F86C9850139006A482
:105B2500E0FF90081EE0D39F500CA3E0C39F400602
:0B5B35009008217401F0900821E0FFAF
:015B40002242
:0B6D1700900849EFF0A3EDF0A3EBF0B3
:106D2200A2AFE433A3F0C2AF12892790084AE0FE73
:106D3200900849E0FDEDFF900851EEF0A3EFF0E47A
:106D420090084DF090084BE0FF900851E0FCA3E062
:106D5200FD7B017A0679BE90086BE4F0A37419F00A
:106D62001285E0900852E02419F0900851E03400B6
:106D7200F090084DE075F019A42400F974E035F0A4
:106D8200FAA374FFF0A3EAF0A3E9F01288FE9008D8
:106D92004EA3E0FAA3E0AE02FF7B017A0679BE9031
:106DA200088AE4F0A37419F012800812854D900845
:106DB2004DE004F0E0C3941E408A7F5E1288B090DA
:076DC200084CE024FF92AF32
:016DC90022A7
:0B4F700090085CEFF0A3EDF0A3EBF065
:104F7B00A2AFE433A3F0C2AF12892790085DE0FE25
:104F8B0090085CE0FDEDFF900861EEF0A3EFF0E41C
:104F9B00900860F0900860E0FFC3941E504C75F0D1
:104FAB0019EFA42400F582E5F034E0AF82FE9008FF
:104FBB0063F0FAA3EFF0FB90085EE0FF900861E06E
:104FCB00FCA3E0FDA9037BFF900873E4F0A3741925
:104FDB00F0128769900862E02419F0900861E034C0
:104FEB0000F0900860E004F080AA7F5E1288B09019
:074FFB00085FE024FF92AF04
:01500200228B
:03000000024000BB
:03000300025003A5
:03000B000250069A
:030013000250098F
:03001B0002500C84
:0300230002500F79
:03002B000250126E
:0300330002501563
:03003B0002501858
:0300430002501B4D
:03004B0002501E42
:0300530002502137
:03005B000250242C
:0300630002502721
:03006B0002502A16
:0300730002502D0B
:03007B0002503000
:03008300025033F5
:03008B00025036EA
:03009300025039DF
:03009B0002503CD4
:0300A30002503FC9
:10400000787FE4F6D8FD9000007F007E20E4F0A3E6
:0A401000DFFCDEFA75812102405545
:10401A0002409AE493A3F8E493A34003F68001F2E2
:10402A0008DFF48029E493A3F85407240CC8C333A7
:10403A00C4540F4420C8834004F456800146F6DF76
:10404A00E4800B0102040810204080906DCAE47ECF
:10405A00019360BCA3FF543F30E509541FFEE4936B
:10406A00A360010ECF54C025E060A840B8E493A332
:10407A00FAE493A3F8E493A3C8C582C8CAC583CA5D
:10408A00F0A3C8C582C8CAC583CADFE9DEE780BE15
:016E79000018
:1047C400E709F608DFFA8046E709F208DFFA803ED7
:1047D40088828C83E709F0A3DFFA8032E309F608C4
:1047E400DFFA8078E309F208DFFA807088828C832C
:1047F400E309F0A3DFFA806489828A83E0A3F608E0
:10480400DFFA805889828A83E0A3F208DFFA804CB9
:1048140080D280FA80C680D4806980F28033801090
:1048240080A680EA809A80A880DA80E280CA8033F9
:1048340089828A83ECFAE493A3C8C582C8CCC58371
:10484400CCF0A3C8C582C8CCC583CCDFE9DEE78041
:104854000D89828A83E493A3F608DFF9ECFAA9F0C0
:10486400EDFB2289828A83ECFAE0A3C8C582C8CC16
:10487400C583CCF0A3C8C582C8CCC583CCDFEADE2F
:10488400E880DB89828A83E493A3F208DFF980CC91
:1048940088F0EF60010E4E60C388F0ED2402B4048A
:1048A4000050B9F582EB2402B4040050AF23234531
:0648B400822390481473FA
:1048BA00BB010689828A83E0225002E722BBFE02FC
:0948CA00E32289828A83E493222F
:1048D300BB010CE58229F582E5833AF583E022509A
:1048E30006E92582F8E622BBFE06E92582F8E222E4
:0D48F300E58229F582E5833AF583E49322FE
:10490000BB010989828A83F8E028F022500327F747
:1049100022BBFE05F8E328F3228A838982F8E49318
:0249200028224B
:10492200BB010FF8E58229F582E5833AF583E02899
:10493200F0225009C58229F8E58226F622BBFE093B
:10494200C58229F8E22582F222F8EA2583F583E975
:0349520093282285
:10495500BB010689828A83F0225002F722BBFE0141
:02496500F3223B
:10496700F8BB010DE58229F582E5833AF583E8F086
:10497700225006E92582C8F622BBFE05E92582C832
:02498700F2221A
:10498900EF8DF0A4A8F0CF8CF0A428CE8DF0A42E42
:02499900FE22FC
:10499B00BC000BBE0029EF8DF084FFADF022E4CC00
:1049AB00F875F008EF2FFFEE33FEEC33FCEE9DECC9
:1049BB00984005FCEE9DFE0FD5F0E9E4CEFD22ED0F
:1049CB00F8F5F0EE8420D21CFEADF075F008EF2F59
:1049DB00FFED33FD4007985006D5F0F222C398FD4A
:0549EB000FD5F0EA22E7
:1049F000C5F0F8A3E028F0C5F0F8E5821582700252
:064A00001583E038F022EE
:104A0600A3F8E0C5F025F0F0E58215827002158363
:064A1600E0C838F0E822C0
:104A1C00BB0110E58229F582E5833AF583E0F5F0D8
:104A2C00A3E0225009E92582F886F008E622BBFEB5
:104A3C000AE92582F8E2F5F008E222E5832AF583FB
:084A4C00E993F5F0A3E99322C0
:104A5400BB010DC58229C582C5833AC5830249F0CD
:104A64005011C58229F808E5F026F618F5F0E5821C
:104A740036F622BBFE11C58229F808E225F0F5F0CE
:104A8400F218E23582F222F8E58229F582E5832ADA
:0D4A9400F58374019325F0F5F0E4933822CA
:104AA100F8BB0111E58229F582E5833AF583E8F047
:104AB100E5F0A3F0225009E92582C8F608A6F02204
:0D4AC100BBFE09E92582C8F2E5F008F222EB
:104ACE00E88FF0A4CC8BF0A42CFCE98EF0A42CFC87
:104ADE008AF0EDA42CFCEA8EF0A4CDA8F08BF0A405
:104AEE002DCC3825F0FDE98FF0A42CCD35F0FCEB64
:104AFE008EF0A4FEA9F0EB8FF0A4CFC5F02ECD3929
:0F4B0E00FEE43CFCEAA42DCE35F0FDE43CFC2295
:104B1D0075F008758200EF2FFFEE33FECD33CDCC4F
:104B2D0033CCC58233C5829BED9AEC99E5829840D2
:104B3D000CF582EE9BFEED9AFDEC99FC0FD5F0D6AF
:104B4D00E4CEFBE4CDFAE4CCF9A88222B800C1B9D9
:104B5D000059BA002DEC8BF084CFCECDFCE5F0CB17
:104B6D00F97818EF2FFFEE33FEED33FDEC33FCEB50
:104B7D0033FB10D703994004EB99FB0FD8E5E4F90B
:104B8D00FA227818EF2FFFEE33FEED33FDEC33FCF8
:104B9D00C933C910D7059BE99A4007EC9BFCE99AEC
:104BAD00F90FD8E0E4C9FAE4CCFB2275F010EF2F31
:104BBD00FFEE33FEED33FDCC33CCC833C810D70731
:104BCD009BEC9AE899400AED9BFDEC9AFCE899F86C
:0E4BDD000FD5F0DAE4CDFBE4CCFAE4C8F922FF
:1080D700C2D5E830E70FB2D5E4C39BFBE49AFAE4D4
:1080E70099F9E498F8EC30E717B2D512810D124BE5
:1080F70059E4C39BFBE49AFAE499F9E498F88003FE
:10810700124B5930D50DE4C39FFFE49EFEE49DFD5D
:04811700E49CFC22C6
:104BEB00EB9FF5F0EA9E42F0E99D42F0EC6480C841
:064BFB0064809845F022E1
:104C0100E8600FECC313FCED13FDEE13FEEF13FF91
:034C1100D8F122B5
:0C4C1400ECF0A3EDF0A3EEF0A3EFF02213
:104C2000A8828583F0D083D082124C37124C371281
:104C30004C37124C37E473E493A3C583C5F0C583A6
:104C4000C8C582C8F0A3C583C5F0C583C8C582C8DE
:014C50002241
:104C5100D083D082F8E4937012740193700DA3A3F2
:104C610093F8740193F5828883E473740293686006
:064C7100EFA3A3A380DF06
:104C7700EF4E6012EF60010EEDBB010B89828A8354
:104C8700F0A3DFFCDEFA2289F05007F709DFFCA961
:0C4C9700F022BBFEFCF309DFFCA9F022B8
:00000001FF
